:100000000C9489000C94A6000C94A6000C94A600F5
:100010000C94A6000C94A6000C94A6000C94A600C8
:100020000C94A6000C94A6000C94A6000C94A600B8
:100030000C94A6000C94A6000C94A6000C946102EB
:100040000C94A6000C94A6000C94A6000C94A60098
:100050000C94A6000C94A6000C94A6000C94A60088
:100060000C94A6000C94A6000C94A6000C94A60078
:100070000C94A6000C94A6000C94A6000C94A60068
:100080000C94A6000C94A6000C94A60049324320C0
:10009000535441525420434F4E444954494F4E20EB
:1000A0004552524F520049324320534C415645204D
:1000B00041444452455353204552524F5200493215
:1000C000432044415441205458204552524F52003D
:1000D0004932432044415441205258204552524F06
:1000E00052004932432054494D454F55540049323E
:1000F00043204552524F520A0020545743523D2547
:10010000303278205354415455533D253032780ACB
:10011000000011241FBECFEFD0E1DEBFCDBF11E044
:10012000A0E0B1E0E4E8FEE000E00BBF02C0079011
:100130000D92A034B107D9F711E0A0E4B1E001C0FD
:100140001D92A934B107E1F70C9485020C940000CC
:1001500084E980937400E4E7F0E0808184FDFDCFC2
:1001600080E090E00895CF92DF92EF92FF920F939C
:100170001F936C01E62E042F0E94A800DF92CF92FD
:100180000E94DA0311271F930F93FF24FF92EF922F
:1001900089EF90E09F938F930E94DA038DB79EB70B
:1001A00008960FB6F8949EBF0FBE8DBF1F910F919A
:1001B000FF90EF90DF90CF900895EF92FF920F9312
:1001C0001F93FC01342F522F1092420110924101D3
:1001D000662321F084EC8093740003C084E880934C
:1001E00074008091740088233CF0809141019091CB
:1001F0004201885E9340A8F38091410190914201B1
:10020000885E9340E0F05523B1F10F2EF1E7EF2E19
:10021000FF24F02DF701408104E710E0F801608130
:1002200080ED90E00E94B300F7014081F801608109
:1002300082EE90E00E94B3008FEF9FEF1EC04091CE
:100240007100842F9927887F9070232F332782177E
:10025000930759F0552379F06091740080ED90E098
:100260000E94B3008FEF9FEF08C0809173008083DE
:1002700080E090E002C08FEF9FEF1F910F91FF9001
:10028000EF900895EF92FF920F931F93542F1092C7
:100290004201109241018093730084E880937400BE
:1002A000E4E7F0E0808188233CF080914101909167
:1002B0004201885E9340B0F38091410190914201E8
:1002C000885E9340E0F0552399F10F2EF1E7EF2E71
:1002D000FF24F02DF701408104E710E0F801608170
:1002E0008EEB90E00E94B300F7014081F80160813D
:1002F00082EE90E00E94B3008FEF9FEF1BC0409111
:100300007100842F9927887F9070262F33278217BA
:10031000930719F480E090E00DC0552349F06091F7
:1003200074008EEB90E00E94B3008FEF9FEF02C04D
:100330008FEF9FEF1F910F91FF90EF900895EF9235
:10034000FF920F931F93342F522F1092420110925D
:100350004101880F862B8093730084E8809374009A
:10036000E4E7F0E0808188233CF0809141019091A6
:100370004201885E9340B0F3809141019091420127
:10038000885E9340E0F0552399F10F2EF1E7EF2EB0
:10039000FF24F02DF701408104E710E0F8016081AF
:1003A00086EA90E00E94B300F7014081F801608185
:1003B00082EE90E00E94B3008FEF9FEF1BC0409150
:1003C0007100842F9927887F9070232F33278217FD
:1003D000930719F480E090E00DC0552349F0609137
:1003E000740086EA90E00E94B3008FEF9FEF02C096
:1003F0008FEF9FEF1F910F91FF90EF900895EF9275
:10040000FF920F931F93282F1092420110924101E7
:1004100084EA80937400E4E7F0E0808188233CF074
:100420008091410190914201885E9340B0F38091A8
:10043000410190914201885E9340E0F0662361F1B2
:100440000F2EF1E7EF2EFF24F02DF701408104E796
:1004500010E0F80160818CE890E00E94B300F701A1
:100460004081F801608182EE90E00E94B3008FEF3E
:100470009FEF14C040917100421719F480E090E0A2
:100480000DC0662349F0609174008CE890E00E94F2
:10049000B3008FEF9FEF02C08FEF9FEF1F910F917F
:1004A000FF90EF9008959C0112BE109242011092AD
:1004B0004101809141019091420182179307C9F750
:1004C00008951F920F920FB60F9211248F939F934E
:1004D0008091410190914201019690934201809355
:1004E00041019F918F910F900FBE0F901F90189513
:1004F00013BE86B7836086BF87B7836087BF8DE0F2
:1005000083BF12BE8DE781BF0895CFEFD0E1DEBF7C
:10051000CDBF0E9478027894E1E7F0E080818C7F83
:1005200080838CE180937000E4E7F0E08081846058
:10053000808380E091E00E9408030E94A80280E08E
:1005400092E00E9453028AE291E00E940803FFCFEA
:10055000CF93DF93CDB7DEB721970FB6F894DEBF08
:100560000FBECDBF8FEF898361E088E00E94FF015D
:10057000882319F08FEF9FEF42C021E048E160E04F
:1005800082E60E949F01882319F08EEF9FEF37C00B
:1005900041E068E280E00E944201882319F08DEF7B
:1005A0009FEF2DC061E080E10E94FF01882319F0D8
:1005B0008CEF9FEF24C021E040E461E082E60E94DE
:1005C0009F01882319F08BEF9FEF19C021E048E5C8
:1005D00060E0CE0101960E94DD00882319F08AEFC9
:1005E0009FEF0DC00E94A800882319F089EF9FEFAC
:1005F00006C08981882309F0B7CF80E090E021967A
:100600000FB6F894DEBF0FBECDBFDF91CF91089536
:100610000F931F93CF93DF93EC0161E088E00E947A
:10062000FF01882319F08FEF9FEFBFC021E048E161
:1006300060E082E60E949F01882319F08EEF9FEF11
:10064000B4C009E311E041E068E2F80180810E9452
:100650004201882309F09BC00F5F1F4FF1E00B336D
:100660001F0789F741E068E2809140010E94420142
:10067000882319F08CEF9FEF98C041E068E28091E9
:1006800038010E944201882319F08BEF9FEF8DC043
:1006900041E068E2809137010E944201882319F00D
:1006A0008AEF9FEF82C00E94A800882319F089EF8B
:1006B0009FEF7BC061E088E00E94FF01882319F072
:1006C00088EF9FEF72C021E048E160E082E60E947F
:1006D0009F01882319F087EF9FEF67C00BE311E0BC
:1006E00041E068E2F80180810E944201882309F01C
:1006F00051C00F5F1F4FF1E00D331F0789F788814D
:10070000882359F041E068E20E944201882309F001
:1007100044C0219688818823A9F741E068E280E0FF
:100720000E944201882319F084EF9FEF3EC00E948F
:10073000A800882319F083EF9FEF37C061E088E0BD
:100740000E94FF01882319F082EF9FEF2EC021E065
:1007500048E160E082E60E949F01882319F081EF62
:100760009FEF23C0CDE3D1E041E068E288810E94A1
:1007700042018823A9F4219681E0CF33D807A1F75D
:100780000E94A800882379F08FEE9FEF0EC08DEFB6
:100790009FEF0BC086EF9FEF08C085EF9FEF05C06E
:1007A00080EF9FEF02C080E090E0DF91CF911F913A
:1007B0000F910895CF93DF93CDB7DEB722970FB691
:1007C000F894DEBF0FBECDBFFE01379661917191E7
:1007D000FA83E983E0914501F091460183818860C5
:1007E000838349815A8180914501909146010E94FD
:1007F0000904E0914501F09146012381277F23837D
:1008000022960FB6F894DEBF0FBECDBFDF91CF9119
:1008100008952F923F924F925F926F927F928F92A4
:100820009F92AF92BF92CF92DF92EF92FF920F937F
:100830001F93CF93DF93CDB7DEB764970FB6F894CD
:10084000DEBF0FBECDBFCC24DD2476011C017C8B26
:100850006B8B2A01FC0117821682838181FD03C004
:100860008FEF9FEF88C2AA24BB2472C2A0FE57C29A
:100870008A8980538A30E8F4FA89F03341F42D856F
:10088000222329F4A3FC03C080E091E06FC08AE03A
:10089000ED85E802C0011124FA89F80FF053FD87B5
:1008A000F7FF02C02FE72D87A3FC4CC23D853E8792
:1008B00049C2C50188709070A3FE05C0ED85EE2386
:1008C00011F4F1E0FD872A89283624F525360CF04D
:1008D0005BC0233509F480C024358CF42B32C1F180
:1008E0002C3234F42032C1F1233209F00DC23CC065
:1008F0003A893D32B1F13E3209F006C23AC08A89E6
:10090000833609F449C084360CF081C0883509F07B
:10091000FBC11BC0EA89E03709F4A3C0E13744F406
:10092000EC3669F1EF3671F0E93609F0EDC16FC0D0
:10093000FA89F53709F49DC0F83739F0F33709F033
:10094000E3C134C028E0298B94C030E1398B91C0D9
:1009500080E190E0A82AB92AE0E2F0E0AE2ABF2ABE
:10096000F1C120E830E00DC080E490E0A82AB92A67
:10097000E9C1E8E0F0E0AE2ABF2A1D86E3C124E029
:1009800030E0A22AB32ADEC14FE3C42E3E853150A7
:100990003E8783E68A8B44C1F201C080FE85F15018
:1009A000FE8722E030E0420E531E3AC1F201C080C1
:1009B000D180892B49F0FD856F2F772767FD7095D2
:1009C000C6010E94E80619C0F60101900020E9F76F
:1009D0003197EC19E98B12C0F201C080D180892BCC
:1009E00049F0FD856F2F772767FD7095C6010E943E
:1009F000DD0603C0C6010E94D406898B22E030E0E8
:100A0000420E531E3E858989381B3E8709C1A2FECE
:100A100008C0F20180819181A281B38124E030E09D
:100A200009C0F20180819181AA2797FDA095BA2F74
:100A300022E030E0420E531E6C017D01B7FF0CC076
:100A400082E090E0A82AB92AF094E094D094C0946F
:100A5000C11CD11CE11CF11CEFEBFFEFAE22BF2249
:100A600021C020E430E0A22AB32A38E73A8B80E1A3
:100A7000898BA2FE08C0F20180819181A281B3819D
:100A800024E030E007C0F20180819181AA27BB27D2
:100A900022E030E0420E531E6C017D018FEC9FEF8F
:100AA000A822B92287017601FE013196F88BEF87E3
:100AB000F9896F2E772488249924C801B701A401ED
:100AC00093010E9420076A3024F02A89620F615244
:100AD00001C0605DEF85F8896193F88BEF87C801ED
:100AE000B701A40193010E94200779018A01211511
:100AF00031054105510509F7CC24DD247601CE01ED
:100B00000196CF84C81AC50182739070892B19F0A1
:100B1000FE85F150FE87A6FE09C02989203111F417
:100B200082E001C081E03E85381B3E8738E0832E9D
:100B3000912C8A209B20A3FE1BC08D85282F332754
:100B400027FD30958C2D99278217930754F0E7EFF6
:100B5000FFEFAE22BF2228E0822E912C8A209B201C
:100B600007C0FD85FC19FD872E852F1B2E8703C02E
:100B70003E853C193E87C50180789170892B69F4C8
:100B80008E8506C0B10180E290E00E94F306812FBD
:100B9000182F11501816B4F31E87A1FE04C0B1011E
:100BA0008DE290E00BC0A4FE04C0B1018BE290E0A6
:100BB00005C0A5FE05C0B10180E290E00E94F306E9
:100BC000A6FE10C0B10180E390E00E94F30689897F
:100BD000803141F4B101EA898E2F992787FD9095E4
:100BE0000E94F306B0FE0DC08E8506C0B10180E301
:100BF00090E00E94F306812F182F11501816B4F3BD
:100C00001E87892869F02D8506C0B10180E390E038
:100C10000E94F306212F122F11501216B4F31D87D4
:100C200090E8692E712C6A207B20A7FC0DC08E8570
:100C300006C0B10180E290E00E94F306812F182FD8
:100C400011501816B4F31E87FA89F33641F4B10136
:100C50008C2D992787FD90950E94F30645C02A891F
:100C60002337B1F446015601198909C0F501819174
:100C70005F01B101992787FD90950E94F3061150FD
:100C8000A8F76401F989CF0ED11C2FEF298B2CC056
:100C90003A89333519F00F8518891FC0460186013E
:100CA000B98808C0F8018491B10199270E94F30620
:100CB0000F5F1F4FBA94FFEFBF16A1F76401298998
:100CC000C20ED11CF98B10C0F80182918F01B101C5
:100CD000992787FD90950E94F306CE01019608178B
:100CE000190791F7188B0F876728B1F08E8506C01A
:100CF000B10180E290E00E94F306812F182F11507D
:100D00001816B4F31E8708C0B101FA898F2F9927EE
:100D100087FD90950E94F306AA24BB2413C02A895C
:100D2000253241F43AE0398B1E861D8681E0A82EDB
:100D3000B12C08C0B101EA898E2F992787FD9095C3
:100D40000E94F3062B893C892F5F3F4F3C8B2B8BF6
:100D5000F101838183FF04C0EB89FC89F49103C016
:100D6000EB89FC89F081FA8B2A89222309F07ECD58
:100D7000F1018681978164960FB6F894DEBF0FBEAD
:100D8000CDBFDF91CF911F910F91FF90EF90DF903A
:100D9000CF90BF90AF909F908F907F906F905F901B
:100DA0004F903F902F900895FC0105900020E9F7A7
:100DB000809590958E0F9F1F0895FC0105906150BE
:100DC00070400110D8F7809590958E0F9F1F089561
:100DD000FC016150704001900110D8F7809590950A
:100DE0008E0F9F1F08950F931F93CF93DF938C0156
:100DF000EB018B81992781FF1BC082FF0DC02E81E3
:100E00003F818C819D812817390764F4E881F9813D
:100E10000193F983E88306C0E885F985802F099559
:100E2000892B31F48E819F8101969F838E8302C02E
:100E30000FEF1FEFC801DF91CF911F910F91089520
:100E4000A1E21A2EAA1BBB1BFD010DC0AA1FBB1FCE
:100E5000EE1FFF1FA217B307E407F50720F0A21B40
:100E6000B30BE40BF50B661F771F881F991F1A94AD
:100E700069F760957095809590959B01AC01BD01D7
:040E8000CF01089501
:100E840057656C636F6D6520746F207468652042CC
:100E940044206D6963726F2053503033207465733E
:100EA400742070726F6772616D0048656C6C6F209E
:100EB400776F726C6421000305000000000040009D
:00000001FF
